:020000040000FA
:06000000852841302A3082
:08000800A000030EA100831209
:100010000C1C2328DD1B23288E015C1C15285C107A
:100020005A088F005D0985051B285C145B088F004A
:100030005D088504DC170C108B180828210E83003E
:10004000A00E200E090005192B2883160117831214
:10005000B23081005D288316011383120B193728F3
:10006000AE17280A03192E17AE1948285628AE13C2
:10007000AE1945282E1F5628AE1A5628A701A601EC
:10008000A501A801AE01AE165D28F030AE055D28D1
:100090002D152E13AE122708AB002608AA0025083E
:1000A000A9002808AC00F030AE055D282E0DA80D83
:1000B000A50DA60DA70DAE1AAE0A8B100B11210EC1
:0800C0008300A00E200E0900D0
:06010A002030840080019A
:10011000840A80300402031C8728682283160C306E
:10012000850587018312850187010730990000301A
:100130009A00103083168E008312603083168F0071
:1001400083120030831691009F008312C8308316FB
:100150008100831201309000013083168C008312DD
:1001600010308B00BD1BB628851DFC223D1BBE0137
:100170003D1BBF013D1FF42281018E018F010B1138
:100180008B100B108C010B178B17D7202D19D92032
:100190003A22B30BD328031085190314BA0DF0309B
:1001A0003A020319B321DC182E233C23C52864002E
:1001B000080029083F3C0319E5282B082A062906D0
:1001C0002C02031D2D11031D08002D110130B70055
:1001D0008B132030370783169B001C141A088312D8
:1001E000A4001030370783169B001C141A088312D2
:1001F000A3000030370783169B001C141A088312D3
:10020000A2008B1724082B02031DAD2923082A0204
:10021000031DAD29013003303702031D3D29290894
:100220003F3C0319272940302906E039031D1D29C9
:100230003F1F1D293F13AD172B2960302906E039D8
:10024000031D2B293F1B2B293F17AD172B29AC1F53
:100250003F13AC1B3F1780302906F039031D3429AA
:10026000BF1F3429BF13AD1790302906F039031D85
:100270003D29BF1B3D29BF17AD17A91FAD29291B5C
:10028000AD2922082906F039A91EE039031DAD2940
:10029000220829050F3903197A2901303702031D75
:1002A00056293E1856293E14AD17822202303702D5
:1002B000031D5F29BE185F29BE14AD1796220330B7
:1002C0003702031D68293E1968293E15AD17AA2279
:1002D00004303702031D7129BE197129BE15AD17EF
:1002E000BE2205303702031D7A293E1A7A293E16AE
:1002F000AD17D222290922050F390319AD29013082
:100300003702031D88293E1C88293E10AD17DC22C8
:1003100002303702031D9129BE1C9129BE10AD1772
:10032000DF2203303702031D9A293E1D9A293E1110
:10033000AD17E22204303702031DA329BE1DA329F5
:10034000BE11AD17E62205303702031DAC293E1E53
:10035000AC293E12AD17EA22AD29B70A06303702A2
:1003600003180800E8280B13DD17B601B301963017
:10037000B4000130B5000130B70085018701AD132D
:100380001F22D720B30BDE29031085190314BA0DE1
:10039000F0303A0203190D2AB41F8501B41F8701FA
:1003A000B40BDE293708B6080319B6000319DC2997
:1003B000FF3085008700B6039630B4002D1DC1299B
:1003C0002D11A91FC129291BC129A91E29120F30CE
:1003D00029050319C129B9012918B90AA918B90AA7
:1003E0002919B90AA919B90AB918C1293919C1298C
:1003F0008B1320303707BC002B08BB00482210307D
:100400003707BC002A08BB00482200303707BC0071
:100410002908BB0048228B17192285018701B70ADA
:10042000B60106303702031CC1290B17DD13F42275
:1004300008000530370203190800850187011430D0
:10044000B90033308F1F85008F1B8501D7202D1DEC
:10045000212A2D11290A0319312AA91F212A291B12
:10046000212A0F302905031D1F2AB90B212A8501D6
:1004700087010800AD1F0800AD131030BC003E0816
:10048000BB0048223030BC003F08BB0048220800B7
:100490003C088B1383169B001C141A0883128B17BD
:1004A0003B02031908008B133B0883161C159A00A6
:1004B00083123C0883169B0055309D00AA309D0096
:1004C0009C1464009C18612A1C1183128B1708006D
:1004D0000A30DE007D30DF00831600309B001C14E4
:1004E0001A088312BD00831610309B001C141A08D2
:1004F0008312BE00831630309B001C141A0883122E
:10050000BF0008000730C100D2100E303E05031DA9
:1005100008008B13831620309B001C141A088312CA
:10052000D6008B178E018F010C1008000630C20018
:1005300052110D303E05031D08008B138316203029
:100540009B001C141A088312D6008B178E018F0192
:100550000C1008000730C300D2110B303E05031DFC
:1005600008008B13831620309B001C141A0883127A
:10057000D6008B178E018F010C1008000530C400C7
:10058000521207303E05031D08008B1383162030DE
:100590009B001C141A088312D6008B178E018F0142
:1005A0000C1008008B13831640309B001C141A0893
:1005B0008312D1008B1708008512DD120800051286
:1005C0005D120800DC1C8510DD100800DC1C051025
:1005D0005D1008008B13831641309B001C141A0811
:1005E0008312D1008B170800C101C201C301C401ED
:1005F0003E1EEA2AD22A0800B601B301B4013D1C0E
:10060000042B3D10BD14112BBD1C092BBD103D1535
:10061000112B3D1D0E2B3D11BD15112BC030BD05FD
:100620003D143D083F39B6006400162B172B182BDC
:10063000192B1A2B3330B41B8500B41F8501B30B63
:10064000142BB40B142B0310B60CB608031D142B7B
:100650000030BC003D08BB0048220800BF1F392BFA
:100660003F1B85103F1B05143F1F85143F1F0510BE
:100670000800851005100800DC10BD18DC14BD1939
:10068000DC145108FF3CDB00F0305107DA000F307A
:100690003E0503190800D6080319572BDC1F080074
:1006A000DC13DF0B08007D30DF00D60308003E1CA2
:1006B000DD123E18DD16BE1C5D12BE185D163E1D15
:1006C000DD10DC18652B3E19DD14BE1D5D10DC1835
:1006D0006B2BBE195D14DC185D10DC18DD10DE0B11
:1006E00008000A30DE00521C8512D21C0512DC18EC
:1006F0007D2B521D8510D21D05103D18842BBD1871
:10070000842B0F30D2000800862308004D08D50046
:10071000E123CD004E08D500E123CE004F08D500DF
:100720004D1CE123CF005008D500CD1CE123D000A3
:10073000C108031952140319A92BC90BA92BCD1BEE
:10074000C1034D08C900CD185214CD1E5210CD1D45
:100750005210C2080319D2140319BA2BCA0BBA2BB0
:10076000CE1BC2034E08CA00CE1AD2144E1DD210A0
:100770004E1FD210BD18E02BBD19E02BC308031982
:1007800052150319CF2BCB0BCF2BCF1BC3034F0815
:10079000CB004F1A52154F1F5211CF1D5211C408D2
:1007A0000319D2150319E02BCC0BE02BD01BC4038B
:1007B0005008CC00501AD215D01FD211D01DD21122
:1007C0000800C001D5080319D50355184014D51ADF
:1007D00040144008C001551C4014D51E4014C005EB
:0607E000C00C550C0800DE
:084000000700000006000200A9
:02400E00CC33B1
:1042000001008100820084008800B100B200B40087
:10421000B800A100A200FF00FF00FF00FF00FF00A8
:104220000000010001000100010001000100010087
:10423000010001000100FF00FF00FF00FF00FF0080
:10424000000000000000000000000000000000006E
:10425000000000000000FF00FF00FF00FF00FF0063
:104260000000FF00FF00FF00FF00FF00FF00FF0055
:10427000FF00FF00FF00FF00FF00FF00FF00FF0046
:1042800002000F00FF00FF00FF00FF00FF00FF0023
:10429000FF00FF00FF00FF00FF00FF00FF00FF0026
:1042A000FF00FF00FF00FF00FF00FF00FF00FF0016
:1042B000FF00FF00FF00FF00FF00FF00FF00FF0006
:1042C000FF00FF00FF00FF00FF00FF00FF00FF00F6
:1042D000FF00FF00FF00FF00FF00FF00FF00FF00E6
:1042E000FF00FF00FF00FF00FF00FF00FF00FF00D6
:1042F000FF00FF00FF00FF00FF00FF00FF00DD00E8
:00000001FF
